:1008380075815F751801751902751A03751B0475A2
:100848001C05751D06751E071208001208867F18FC
:0A0858007D071208A812080080EEC8
:1008C600E4FDFCC3ED9FEC9E50070DBD00010C80BE
:0108D600F22F
:0108D70022FE
:10080000D287D2867F027E001208C6D287C286C2F5
:10081000A4C2A5C2A6C2A71208C6D287C286C2A415
:10082000C2A5C2A6D2A71208C6D287C286C2A4C2D7
:08083000A5C2A6C2A70208C67A
:10088600D287C286D2A4C2A5C2A6D2A77F027E0004
:100896001208C6D287C286D2A4C2A5C2A6C2A70221
:0208A60008C682
:0408A800AB07A905EC
:1008AC00E4FAEAC399501275A0007F707E17120803
:0908BC00C6D287D2860A0B80E93E
:0108C5002210
:0908E400759024D28875A88122C8
:030003000208628E
:07086200C0E0C0D075D00812
:1008690075815F75903F75901FE590540FFFAE102D
:08087900051074112EF8A60F02
:05088100D0D0D0E032F0
:030000000208D81B
:0C08D800787FE4F6D8FD75811E02083818
:00000001FF
